:030000000208DB18
:0C08DB00787FE4F6D8FD758153020922F5
:1009CA000000415445300D0A0000000000000000FC
:1009DA00000000000000000000000000000000000D
:1009EA0041542B43495053544152543D225443508D
:1009FA00222C223139322E3136382E322E313038ED
:100A0A00222C383038300D0A0041542B43495053B8
:080A1A00454E443D350D0A0074
:100A6700C103C102C1051E360000000000000000DE
:100A7700000000000000000000000000000000006F
:100A8700000000000000012600013500C100C1017F
:030A970001250036
:070B5C0053A27F43A2802297
:040B630053A27F22F8
:0E0B280000007F7F7EE97D94DDFEDEFCDFFABB
:010B3600229C
:0E0B370000007F167E037DE3DDFEDEFCDFFAAC
:010B4500228D
:080B53007F0B7EF6DEFEDFFCE5
:010B5B002277
:100AF00053877F759850438E40538EFE53890F4322
:0D0B00008920758BFD758DFDC2ABD28E2254
:100AC700200203300522120B637B007A007936126D
:100AD7000A9B7E007F1E7D007B007A007936120A12
:090AE7003BC202C205120B5C22A5
:10096700E4FFC206C207120B28120B28120B28122B
:100977000AF0F59175923FD2ACD2AFD29C120B5CC4
:10098700120B53120B53FFEF04FE74272FF8A60622
:100997000FBF0DF320060ED2067BFF7A0979CC1222
:1009A7000A9B120B28120AC7300613200710D2071A
:1009B7007BFF7A0979EA120A9B120B28D203120AE3
:0309C700C780D115
:03002300020800D0
:09080000C0E0C0D075D000C000BA
:100809002098030208CDC298E521640D7026E59968
:10081900B40A21E5266401601B20031874372526D4
:10082900F87600D20275260075220075210075231D
:1008390000752400E521B43A14E522B4350FE52307
:10084900B42C0AE524B44405D201752505300125E7
:10085900D3E52564809480400415258018743725D4
:1008690026F876CAD2027526007522007521007510
:100879002300752400C29874362526F8A69985990F
:1008890021D3E52664809480400874352526F8E64E
:10089900F522D3E52664809481400874342526F82E
:1008A900E6F522D3E526648094824008743425262F
:1008B900F8E6F5220526D3E5266480949D40057562
:0B08C9002600D205309904C299C20439
:0708D400D000D0D0D0E032CB
:0D0B460030040122EFD204F5992004FD22B5
:100A9B008B0B8A0C890DAB0BAA0CA90D120A2260C9
:100AAB001A120B53AB0B050DE50DAA0C7002050CBE
:0C0ABB0014F9120A22FF120B4680DB2205
:100B0D008B088A09890A7BFF7A0A7913120A9B12CC
:0B0B1D000B28AB08AA09A90A020A9BDA
:1008E700020967E493A3F8E493A34003F68001F2B7
:1008F70008DFF48029E493A3F85407240CC8C33312
:10090700C4540F4420C8834004F456800146F6DFE0
:10091700E4800B0102040810204080900A67E47EFF
:10092700019360BCA3FF543F30E509541FFEE493D5
:10093700A360010ECF54C025E060A840B8E493A39C
:10094700FAE493A3F8E493A3C8C582C8CAC583CAC7
:10095700F0A3C8C582C8CAC583CADFE9DEE780BE7F
:010A9A00005B
:100A2200BB010689828A83E0225002E722BBFE02D2
:090A3200E32289828A83E4932205
:100A3B00EF4E6012EF60010EEDBB010B89828A83D2
:100A4B00F0A3DFFCDEFA2289F05007F709DFFCA9DF
:0C0A5B00F022BBFEFCF309DFFCA9F02236
:00000001FF
